 adcsdk

 Timestamp is 4da293a6 (Mon Apr 11 17:37:42 2011)

 Preferred load address is 10000000

 Start         Length     Name                   Class
 0001:00000000 00000004H .CRT$XCA                CODE
 0001:00000004 00000004H .CRT$XCZ                CODE
 0001:00000008 00000004H .CRT$XIA                CODE
 0001:0000000c 00000004H .CRT$XIZ                CODE
 0001:00000010 00000004H .CRT$XPA                CODE
 0001:00000014 00000004H .CRT$XPZ                CODE
 0001:00000018 00000004H .CRT$XTA                CODE
 0001:0000001c 00000004H .CRT$XTZ                CODE
 0001:00000020 0000003cH .rdata                  CODE
 0001:0000005c 00000023H .rdata$debug            CODE
 0001:00000080 00000618H .text                   CODE
 0001:00000698 00000014H .idata$2                CODE
 0001:000006ac 00000014H .idata$3                CODE
 0001:000006c0 0000002cH .idata$4                CODE
 0001:000006ec 0000000cH .idata$6                CODE
 0001:00000700 0000008fH .edata                  CODE
 0002:00000000 0000002cH .idata$5                DATA
 0002:0000002c 0000003cH .data                   DATA
 0002:00000068 00000010H .bss                    DATA
 0003:00000000 00000060H .pdata                  DATA

  Address         Publics by Value              Rva+Base       Lib:Object

 0000:00000000       ___safe_se_handler_count   00000000     <absolute>
 0000:00000000       ___safe_se_handler_table   00000000     <absolute>
 0001:00000000       __xc_a                     10001000     corelib0:crt0init.obj
 0001:00000004       __xc_z                     10001004     corelib0:crt0init.obj
 0001:00000008       __xi_a                     10001008     corelib0:crt0init.obj
 0001:0000000c       __xi_z                     1000100c     corelib0:crt0init.obj
 0001:00000010       __xp_a                     10001010     corelib0:crt0init.obj
 0001:00000014       __xp_z                     10001014     corelib0:crt0init.obj
 0001:00000018       __xt_a                     10001018     corelib0:crt0init.obj
 0001:0000001c       __xt_z                     1000101c     corelib0:crt0init.obj
 0001:0000003c       ??_C@_1BE@FABCBOME@?$AAM?$AAU?$AAT?$AAE?$AAX?$AA_?$AAA?$AAD?$AAC?$AA?$AA@ 1000103c     adcsdk_common_topaz_v1:adc_sdk.obj
 0001:00000050       ??_C@_1M@EPBPGMBG@?$AAA?$AAD?$AAC?$AA1?$AA?3?$AA?$AA@ 10001050     adcsdk_common_topaz_v1:adc_sdk.obj
 0001:00000080       AdcInit                    10001080 f   adcsdk_common_topaz_v1:adc_sdk.obj
 0001:00000118       AdcDeinit                  10001118 f   adcsdk_common_topaz_v1:adc_sdk.obj
 0001:00000160       AdcConfigureChannel        10001160 f   adcsdk_common_topaz_v1:adc_sdk.obj
 0001:0000024c       AdcGetSamples              1000124c f   adcsdk_common_topaz_v1:adc_sdk.obj
 0001:000003ec       DllEntry                   100013ec f   adcsdk_common_topaz_v1:adc_sdk.obj
 0001:00000400       CloseHandle                10001400 f   coredll:COREDLL.dll
 0001:00000410       CreateMutexW               10001410 f   coredll:COREDLL.dll
 0001:00000420       CreateFileW                10001420 f   coredll:COREDLL.dll
 0001:00000430       ReleaseMutex               10001430 f   coredll:COREDLL.dll
 0001:00000440       DeviceIoControl            10001440 f   coredll:COREDLL.dll
 0001:00000450       WaitForSingleObject        10001450 f   coredll:COREDLL.dll
 0001:00000460       DisableThreadLibraryCalls  10001460 f   coredll:COREDLL.dll
 0001:00000470       _DllEntryCRTStartup        10001470 f   corelib0:pegdentry.obj
 0001:00000574       _cexit                     10001574 f   corelib0:cexit.obj
 0001:00000584       _initterm                  10001584 f   corelib0:crt0dat.obj
 0001:000005b0       _cinit                     100015b0 f   corelib0:crt0dat.obj
 0001:00000610       __security_init_cookie     10001610 f   corelib0:seccinit.obj
 0001:0000065c       __crt_ExitProcess          1000165c f   corelib0:exitproc_proxy.obj
 0001:00000668       free                       10001668 f   corelib1:COREDLL.dll
 0001:00000678       __security_gen_cookie2     10001678 f   corelib1:COREDLL.dll
 0001:00000688       TerminateProcess           10001688 f   coredll:COREDLL.dll
 0001:00000698       __IMPORT_DESCRIPTOR_COREDLL 10001698     coredll:COREDLL.dll
 0001:000006ac       __NULL_IMPORT_DESCRIPTOR   100016ac     coredll:COREDLL.dll
 0002:00000000       __imp_CloseHandle          10002000     coredll:COREDLL.dll
 0002:00000004       __imp_CreateMutexW         10002004     coredll:COREDLL.dll
 0002:00000008       __imp_CreateFileW          10002008     coredll:COREDLL.dll
 0002:0000000c       __imp_ReleaseMutex         1000200c     coredll:COREDLL.dll
 0002:00000010       __imp_DeviceIoControl      10002010     coredll:COREDLL.dll
 0002:00000014       __imp_WaitForSingleObject  10002014     coredll:COREDLL.dll
 0002:00000018       __imp_DisableThreadLibraryCalls 10002018     coredll:COREDLL.dll
 0002:0000001c       __imp_free                 1000201c     corelib1:COREDLL.dll
 0002:00000020       __imp___security_gen_cookie2 10002020     corelib1:COREDLL.dll
 0002:00000024       __imp_TerminateProcess     10002024     coredll:COREDLL.dll
 0002:00000028       \177COREDLL_NULL_THUNK_DATA 10002028     coredll:COREDLL.dll
 0002:00000060       __security_cookie          10002060     corelib0:seccinit.obj
 0002:00000064       __security_cookie_complement 10002064     corelib0:seccinit.obj
 0002:0000006c       _exitflag                  1000206c     corelib0:cexit.obj
 0002:00000070       __onexitend                10002070     <common>
 0002:00000074       __onexitbegin              10002074     <common>

 entry point at        0001:00000470

 Static symbols

 0001:000004b4       doexit                     100014b4 f   corelib0:cexit.obj
